:100000000C9489050C94691B0C94D0050C94D005B4
:100010000C94D0050C94D0050C94D0050C94D0050C
:100020000C94D0050C94D0050C94F72E0C94CB2F87
:100030000C9477280C94D0050C94D0050C94D00522
:100040000C94D0050C94D0050C94D0050C94D005DC
:100050000C94D0050C94CE280C94D0050C94D005AB
:100060000C94D0050C94D0050C94D0050C94D005BC
:100070000C94D0050C94D0050C94D0050C94D005AC
:100080000C94D0050C94D0050C94D0050C94D0059C
:100090000C94D0050C94D0050C94D0050C94D0058C
:1000A0000C94D0050C94D0050C94D00529001400B4
:1000B0001A000800150017002B00040016000700A6
:1000C00009000A00E1001D001B00060019000500E0
:1000D000E000E300E2004C0001512C00A8001300F6
:1000E00012000C0018001C00280033000F000E0046
:1000F0000D000B00E500380037003600100011003D
:100100002D00340030002F0002512A0035001E005F
:100110001F00200021002200010001000100520008
:100120000100010001000100500051004F000100DA
:100130000100010001000100015101000100270040
:1001400026002500240023000100010023002200D6
:10015000210001000100310020001F001E000100ED
:100160002E00310037002700270001003A003B0035
:100170003C003D003E003F00C55CC75CC95CC35C01
:1001800001000100C65CC85CCA5CC45C0100C25CC2
:1001900001000100010001000100010045004400D0
:1001A0004300420041004000010001000100010045
:1001B00001000100010052000100010001000100E6
:1001C0004F005100500001000251010000000000EA
:1001D000000000000000000000000000000000001F
:1001E000000000000000000000000000000000000F
:1001F00000000000000000000000000000000000FF
:1002000000000000000000000000000000000000EE
:1006A0000000000000000000000000000100010048
:1006B0000100010001000100010001000100010032
:1006C0000100010001000100010001000100010022
:1006D0000100010001000100010001000100010012
:1006E0000100010001000100010001000100010002
:1006F00001000100010001000100010001000100F2
:1007000001000100010001000100010000000000E3
:10071000000000002A2B280000000000000000005C
:100720000000000000000029000000002C1E342002
:10073000212224342627252E362D3738271E1F2028
:100740002122232425263333362E37381F0405066D
:100750000708090A0B0C0D0E0F10111213141516B1
:100760001718191A1B1C1D2F3130232D35040506AF
:100770000708090A0B0C0D0E0F1011121314151691
:100780001718191A1B1C1D2F3130354C00000000A2
:100790000000000000000000000000000000000059
:1007A0007E0F00D4FFFFFFC70000007832190A0057
:1007B000047F3F1F643214643214783C1E1E140AF6
:1007C000052223252628292A2C2D2F303233353691
:1007D000383A3B3D3E4042434547494A4C4E5051D2
:1007E000535557595A5C5E6062646668696B6D6FF9
:1007F00071737577797B7D7F81838587898A8C8EFC
:1008000090929496989A9C9E9FA1A3A5A7A8AAAC03
:10081000AEAFB1B3B4B6B8B9BBBCBEBFC1C2C3C53D
:10082000C6C7C9CACBCCCDCED0D1D2D2D3D4D5D6DF
:10083000D7D7D8D9D9DADADBDBDBDCDCDCDCDCDD12
:10084000DDDDDDDCDCDCDCDCDBDBDBDADAD9D9D8F6
:10085000D7D7D6D5D4D3D2D2D1D0CECDCCCBCAC98E
:10086000C7C6C5C3C2C1BFBEBCBBB9B8B6B4B3B1BD
:10087000AFAEACAAA8A7A5A3A19F9E9C9A98969458
:1008800092908E8C8A89878583817F7D7B7977752D
:1008900073716F6D6B6968666462605E5C5A59570C
:1008A000555351504E4C4A4947454342403E3D3BCB
:1008B0003A3836353332302F2D2C2A292826252355
:1008C00022FFAA7F554000010203040506070F0E10
:1008D0000D0C0B0A090800010101010101010101D0
:1008E00002020202020202020203030303030303E1
:1008F00003040404040404040505050505060606AE
:100900000606070707070708080808090909090A6A
:100910000A0A0B0B0B0C0C0C0D0D0D0E0E0E0F0F0F
:100920000F1010111111121213131414151516169D
:100930001717181819191A1A1B1B1C1D1D1E1E1F0C
:100940002020212222232424252626272829292A5B
:100950002B2C2D2D2E2F3031323233343536373883
:10096000393A3B3C3D3E3F4041424344454647487F
:10097000494A4C4D4E4F50515354555658595A5B55
:100980005D5E5F616264656668696B6C6D6F7072F5
:10099000737577787A7B7D7E8082838587888A8C61
:1009A0008E8F91939596989A9C9EA0A2A3A5A7A995
:1009B000ABADAFB1B3B5B7BABCBEC0C2C4C6C9CB8C
:1009C000CDCFD1D4D6D8DBDDDFE2E4E7E9EBEEF042
:1009D000F3F5F8FAFDFF0403300000001C03660085
:1009E0006C00750078006C006100620020007A00E5
:1009F00070006C00690074000000100366006C0059
:100A0000750078006C0061006200000004030904B6
:100A100009025B00030100A0FA09040000010301C0
:100A2000010009211101000122400007058103088E
:100A3000000A09040100020300000009211101005D
:100A4000012222000705820320000107050303207D
:100A50000001090402000103000000092111010046
:100A6000012232000705840320000A120110010050
:100A7000000008767001000100010203010660FF1A
:100A80000961A1010962150026FF00952075088102
:100A9000020963150026FF00952075089102C00524
:100AA000010980A101850319012AB700150126B7A4
:100AB00000950175108100C0050C0901A101850494
:100AC00019012AA002150126A002950175108100C6
:100AD000C005010906A101050719E029E715002550
:100AE00001950875018102950175088101050719B5
:100AF0000029FF150026FF009506750881000508EE
:100B0000190129059505750191029501750391015A
:100B1000C00011241FBECFEFDAE0DEBFCDBF04B6A8
:100B200003FE27C08091540390915503A091560372
:100B3000B09157038730904BA740B04BD1F410923F
:100B4000540310925503109256031092570314BE8B
:100B500084B7877F84BF0FB6F894A8958091600012
:100B6000886180936000109260000FBEE0E0F8E3BF
:100B7000099511E0A0E0B1E0E6E4F6E602C00590D8
:100B80000D92A03FB107D9F723E0A0EFB1E001C07B
:100B90001D92A435B207E1F70E94AD2B0C94D2321E
:100BA0000C9400000F9300E122E041E00E94E9066E
:100BB0000F9108958AEA611101C089EA0C94871E99
:100BC00081E0089581E008950C94E20508950C9465
:100BD000E6051F93CF93DF9300D000D00F92CDB7DF
:100BE000DEB749835A836B833091800289819A8171
:100BF00031111DC06623B9F02223A9F00E94E2251D
:100C0000182F682F89819A810E948B2569817A81AA
:100C1000812F0F900F900F900F900F90DF91CF9139
:100C20001F910C94EF170E94B925182FEFCF0E9447
:100C3000E22569817A81EDCFFC01262F4081518127
:100C40006281738184810C94E905CF93DF93EC0179
:100C500060E00E941C06BE01DF91CF910C94E70575
:100C6000FF920F931F93CF93DF93E82FF0E0E45FA1
:100C7000F84FF490C82FC695C695C695D0E0FE01F2
:100C8000E456F84F0491877010E0082E02C01595C5
:100C900007950A94E2F701701127C457D84FFE0157
:100CA000C491D0E002C0D595C7958A95E2F7C1708E
:100CB000DD270115110519F081EE0E94A91D20976D
:100CC00019F086EE0E94A91D8F2D0E94871ECD2B44
:100CD00019F086EE0E94381E012B41F081EEDF9163
:100CE000CF911F910F91FF900C94381EDF91CF91FF
:100CF0001F910F91FF900895EF92FF920F931F9312
:100D0000CF93DF93EC01162F0AE08881882309F442
:100D100056C0813009F050C08981813061F47E0174
:100D200022E0E20EF11CCA818C2F0E94A91D8C2F9B
:100D30000E94381E09C0823099F47E0182E0E80EDC
:100D4000F11C8A810E94A91DE7012196812F815003
:100D5000E0F2EFE9FFE03197F1F700C00000F7CFD4
:100D6000833031F47E01E2E0EE0EF11C8A81E0CFA7
:100D7000843011F02196E9CF2A81229690E080E01C
:100D8000AE014F5F5F4F2053330B2A30310548F0DF
:100D90000197D8F2EFE9FFE03197F1F700C00000CA
:100DA000F7CF089FB001099F700D1124C901860F6C
:100DB000971F2981EA01E4CF0E943006C6CFDF9158
:100DC000CF911F910F91FF90EF90089560E00C94E8
:100DD0007C068F929F92AF92BF92CF92DF92EF925A
:100DE000FF920F931F936B017C0181E090E0A0E0E4
:100DF000B0E04C015D0104C0880C991CAA1CBB1C0E
:100E00004A95D2F7B501A4014C015D0104C0880CDC
:100E1000991CAA1CBB1C2A95D2F7482959296A2972
:100E20007B2904C0880F991FAA1FBB1F0A95D2F700
:100E30008A019B010C211D212E213F21041715073A
:100E40002607370789F48C299D29AE29BF29BC01C3
:100E5000CD011F910F91FF90EF90DF90CF90BF9049
:100E6000AF909F908F90089580959095A095B095A4
:100E70008C219D21AE21BF21EACF0F93382F262F41
:100E80006091D7027091D8028091D9029091DA02D4
:100E9000042F432F0E94E9060F910C94C9240E944D
:100EA00018290E942C27811102C00E94C9270E9484
:100EB0006C140C94B9090E94C9140C94BC090895CF
:100EC0000C945F0781E008950C946207CF93C82FBC
:100ED0000E9460078C2FCF910C94640708950E94A4
:100EE000F7200E946E072FEF84E39CE021508040A2
:100EF0009040E1F700C000000C94F2280F931F937C
:100F0000CF93DF93EC0161E00E941C068C01BE01CF
:100F10000E94C415882389F1BE01C8010E94E4051E
:100F2000882359F1BE01C8010E942719882329F19D
:100F3000BE01C8010E9468198823F9F0BE01C801EA
:100F40000E948B1A8823C9F0BE01C8010E94BC13FD
:100F5000882399F08A81882339F001158CE51807D8
:100F600051F00E3D1C4579F0CE01DF91CF911F91DC
:100F70000F910C94E0050E946F0780E0DF91CF9104
:100F80001F910F9108950E94C927F7CF90E080E04C
:100F900008950895FC01EE0FFF1FE455F84F859169
:100FA00094910895CF93DF930E94EF170E94DE087B
:100FB000EC01811520E5920708F041C0811530E46D
:100FC000930708F0B4C0803E910518F5803C910568
:100FD00008F09DC0883A910570F4853A910508F0B3
:100FE0008EC081309105F9F00097E9F00497D8F4AC
:100FF000D0E0C0E018C08F3B9105D0F7C85AD0E0D0
:10100000CC0FDD1FCA5CDE4F0990D881C02DD4649F
:101010000AC08115904258F4C11581E0D80718F430
:10102000C83ED10528F7CE01DF91CF910895C115B3
:1010300090E3D90708F071C0CE019F706AC0811596
:1010400025E5920758F5811534E5930708F09EC011
:10105000811542E5940750F4C11581E5D80708F4DD
:1010600069C0DC2FCC27C16FD06ADDCF982F969551
:1010700096959E0123703327C115D34508F077C09C
:10108000C1E0D0E002C0CC0FDD1F2A95E2F720E2DC
:10109000929FC0011124C82BD92B67C0C11589E5C7
:1010A000D807A8F4C11598E5D90708F074C0C11590
:1010B00026E5D20708F09CCF8C2F0E947509C82F17
:1010C000D0E0DC2FCC27CC27DF71D062ACCFC115AC
:1010D0003AE5D30708F464C0CE01905681159042DA
:1010E00008F086CF8D2F8F710E94750990E0982FA0
:1010F000882788279F719C012C2BE901E6CFC55AD0
:10110000D0E0CC59DE4FC881D0E0D0648CCF805C79
:1011100091090E94CA07EC0186CFCE019927D3FF1F
:1011200003C0EC01D86C7FCFEC01D06C7CCFDF70BA
:10113000D06A79CFCE01E4E096958795EA95E1F7FC
:1011400083702C2F26952695237090E2299F90017D
:101150001124382B8C2F8370C1E0D0E002C0CC0F5B
:10116000DD1F8A95E2F7C22BD32BDC685CCFC1E090
:10117000D0E002C0CC0FDD1F2A95E2F730E2939F4A
:10118000C0011124C82BD92BDA684DCFD82FCC271A
:10119000C46FD06A48CFDC2FCC27C06FD06A43CF52
:1011A0008C2F8F700E94750934E0D695C7953A95BB
:1011B000E1F7CF709C2FEC01D06935CF82389105D3
:1011C000B1F1B0F48133910509F475C048F4893266
:1011D000910509F469C08A32910509F473C0089534
:1011E0008533910509F459C08933910501F10895BA
:1011F000833E9105A9F138F4803E9105F9F0823ED5
:10120000910549F10895863E9105A9F1873E910522
:10121000C9F1843E910519F52091460321FF1FC0B5
:101220008091450384FD14C087EE90E008952091DD
:1012300045032370A1F080EE90E0089520914503CE
:1012400020FD47C03091460330FF09C024FF44C051
:1012500090E080E004C02091450322FDF7CF08957F
:101260002091450322FD3BC03091460330FDE3CF82
:1012700024FFF5CFEDCF2091450323FFF0CF24FDD0
:10128000E7CFD2CF2091450323FD2CC030914603F8
:1012900031FFEECF84EE90E008952091450325FFC5
:1012A000DECF89E290E008952091450325FFD7CF56
:1012B00085E390E008952091450326FFD0CF8AE290
:1012C00090E008952091450326FFC9CF81E390E087
:1012D000089589E390E0089583EE90E0089582EE0A
:1012E00090E0089586EE90E008959091450392FF76
:1012F00006C0282F28712830F9F4877F846093FF77
:1013000006C0282F28712831F1F4877E846120914E
:10131000460320FF06C0382F38713830D9F4877F54
:10132000816021FF06C0282F28712831D1F4877EE3
:10133000816194FD877E0895282F24712430F9F669
:101340008B7F8860DCCF282F2471243101F78B7EBE
:101350008861DDCF382F3171313019F78E7F886089
:10136000E0CF282F2171213121F78E7E8861E1CFD6
:1013700008950C94B80908950C94BB09E82FF0E087
:10138000EE5FFC4F80810895089580EA8A95F1F719
:10139000089508950E94480B8091040180910401F2
:1013A00094E0811190E090930B0384E0891B80937B
:1013B0000A03ADE6B1E061E070E08D91E82FE295BF
:1013C000EF70F0E041A18F709B0101C0220F8A9560
:1013D000EAF7922F9095942391A382A1822B82A366
:1013E00081E0A137B80749F7A7E6B1E061E070E016
:1013F0008D91E82FE295EF70F0E041A18F709B0195
:1014000001C0220F8A95EAF7922F9095942391A319
:1014100082A1822B82A381E0AD36B80749F7EAEFBB
:10142000F2E0A2E0B3E082E093E011921D928E1709
:101430009F07D9F784E00E94E50A0E944F070C94A9
:101440005D0B0E94320B8823F1F080910A0390E03B
:101450008E5F9C4F0E948D0B811112C08091F00114
:101460008F5F8093F001863048F0E0910A03F0E04E
:10147000EE5FFC4F10821182128213820C945B0784
:101480001092F001FBCF80910B0390E08E5F9C4F98
:101490000E94AE0B0E94C9140C94C9092F923F926E
:1014A0005F926F927F928F929F92AF92BF92CF92F4
:1014B000DF92EF92FF920F931F93CF93DF930AEF88
:1014C00012E09DE6892E91E0992E2EEFA22E22E0C9
:1014D000B22E712CCC24C394D12CD8015C90F8018D
:1014E00011928F01D4018D914D01C82FC295CF70FB
:1014F000D0E099A18F70760101C0EE0C8A95EAF7D1
:10150000892F8E2989A38AA16E2C609486218AA3B3
:101510000E94C50987E6282E81E0382E30E020E0C1
:10152000F8013197D1014D911D01842F82958F7063
:1015300090E0DC0190968C91608190E04F7002C049
:10154000959587954A95E2F780FD3DC08C2D022E3A
:1015500001C0880F0A94EAF7862B80832F5F3F4FE4
:1015600026303105F9F689A1682269A28AA1E82A04
:10157000EAA281E09081951101C080E0782AA0164E
:10158000B10609F0AACF60910B0370E06E5F7C4F4B
:10159000272D44E08AEF92E00E94E60A0E94210A89
:1015A000872DDF91CF911F910F91FF90EF90DF90EA
:1015B000CF90BF90AF909F908F907F906F905F90F3
:1015C0003F902F90089580E0C7CF0895FF920F932A
:1015D0001F93CF93DF93F82E092F162FD72FC42FE9
:1015E000222349F081E08093F3010E94A728909381
:1015F000F2018093F1018091F3018823A1F08091A1
:10160000F1019091F2010E94BF28069760F0EF2D42
:10161000F02FA12FBD2FCE0FDF2FD11DEC17FD070F
:1016200041F41092F301DF91CF911F910F91FF9040
:10163000089581918D93F2CF82E39091E30097FD1D
:101640000FC0EFE3FCE93197F1F700C000008150D3
:10165000A1F78091D8008F768093D80080E008951C
:1016600081E008958091F401811107C00E941C0B54
:1016700081110AC082E08093F40181E09091F4012D
:10168000913009F080E0089581E0F5CF0C94320BA1
:101690000E94460B809304018091040168E0882336
:1016A00049F080E00E945A0C0E94320B882321F0FE
:1016B0000C94640B88E0F6CF08950E94320B8111E0
:1016C00002C00C946A0B089562E070E085E091E03E
:1016D0000C94161B62E070E085E091E00C941F1BF7
:1016E0000E947B11882361F08CEF91E00E948111B0
:1016F00081E090E00E94F81B892B11F40C947E117C
:1017000008958091FB01883039F460E08CEF91E01E
:101710000E9499121092FB010895CF93DF93D82F66
:10172000C92F0E94700B90E080E00E94F81B009788
:1017300099F4ED2FFC2FDC01AA50BE4F2C91219380
:10174000019684309105B9F78AEF91E00E943A152D
:1017500081E0DF91CF91089580E0FBCFCF93DF93BD
:10176000D82FC92F0E94810BED2FFC2F90E080E035
:101770002191DC01AA50BE4F2C9301968430910533
:10178000B9F78AEF91E0DF91CF910C943115AF92C8
:10179000BF92CF92DF92FF920F931F93CF93DF936D
:1017A000362F472FE82FF0E0EA52F74F71110DC0A6
:1017B0006491762F862FDF91CF911F910F91FF902B
:1017C000DF90CF90BF90AF900895C72FD0E02491C5
:1017D000F22E022F10E056E0659FC0011124EFEFBA
:1017E000F0E0BF010E948931832F90E0880F991F9C
:1017F00035E5369FD001379FB00D11248A1B9B0B16
:10180000982F990F980F6F01CC1ADD0AC09ED00156
:10181000C19EB00DD09EB00D11248B2F949FA001BE
:101820001124452F55276F01C41AD50AC09EA00167
:10183000C19E500DD09E500D11245F01A91AB10810
:10184000AC9E6001AD9ED00CBC9ED00C1124CD2C62
:10185000DD24EC19FD09E09FE001E19FD00DF09F30
:10186000D00D1124ED2F62307105A1F048F46115FF
:10187000710569F06130710589F0EB2F852F07C084
:101880006430710571F088F066307105B1F76E2F24
:10189000722F91CFE22F2B2F8D2FF9CFE22F252FF3
:1018A000F6CFEB2F822F2D2FF2CF2B2F8F2DE52F61
:1018B000EECF0895E7E1F1E0808361830895CF934F
:1018C000DF93762FE901682F842F0E94C70B79835D
:1018D00068838A83DF91CF91089580910C03982FBC
:1018E0009E7F29F48170826080930C030895863571
:1018F000E8F381708465F8CF88E090E00C942F3293
:10190000CF92DF92EF92FF926B017C010E946D0CEF
:10191000B701A60188E090E0FF90EF90DF90CF90B4
:101920000C944D3260910C0370910D0380910E0365
:1019300090910F030C94800CECE0F3E083E0808343
:1019400011828FEF828383831482A1E6B2E0129624
:101950008C911297836012968C9360817181828141
:1019600093810C94800C80910C0380FF02C08695BB
:10197000089580E0089580911003833018F48F5FFC
:101980008093100360910C0370910D0380910E03FE
:1019900090910F030C94800C80911003882319F010
:1019A00081508093100360910C0370910D0380911E
:1019B0000E0390910F030C94800C809110030895F6
:1019C00080931003662351F060910C0370910D0316
:1019D00080910E0390910F030C94800C089560E0A9
:1019E0000C94E00C80910D03089580910E030895EE
:1019F00080910F03089570E00C946714CF92DF92EA
:101A0000EF920F931F93CF93DF93CDB7DEB7E0979D
:101A10000FB6F894DEBF0FBECDBF60911801809164
:101A20000C0380FF36C0E6ECF8E09E012F5F3F4FCD
:101A30008E010F5C1F4FC901A4914A2F50E0DA01BB
:101A4000AA0FBB1FA40FB51FAF5EBC4FCD90DD909A
:101A5000EC90D901CD92DD92ED929D013196A017C7
:101A6000B10751F720911701B3E02B9F800D911D15
:101A700011240E94FB0CE0960FB6F894DEBF0FBE57
:101A8000CDBFDF91CF911F910F91EF90DF90CF905D
:101A900008958091190190911A0123E0829FF0012D
:101AA0001124EF5EFC4F891708F0BDCF1182108220
:101AB00012828F5F3396F7CF90910C0390FF14C082
:101AC0009091190120911A0133E0939FF0011124A4
:101AD000EF5EFC4F921710F00C94FE0C8183608334
:101AE00042839F5F3396F6CF0895CF93DF9300D064
:101AF0000F92CDB7DEB790910C0390FF0AC09E0104
:101B00002F5F3F4F0E945F0C4B8169818A810E9449
:101B10005C0D0F900F900F90DF91CF910895CF93B0
:101B2000DF93EC01EC81F0E0EF53F84F4491ECE0EF
:101B3000F3E0628181810E94750D8C818F5F8C83BF
:101B4000DF91CF910895CF93DF93EC01ECE0F3E0C8
:101B5000438162818C810E94750D8C818F5F8C83A3
:101B6000DF91CF9108950F931F93CF93DF9300D010
:101B70000F92CDB7DEB78C018091040281110AC0AB
:101B80009E012F5F3F4F4FEF6FEF0E945F0C8A81E6
:101B900080930402F8016481613069F0809104024D
:101BA00040E0662361F040E0623011F440910402AD
:101BB00080E060E004C06091040240E080E00E94A8
:101BC0005C0DF801848190E0019663E070E00E9472
:101BD0009D3184830F900F900F90DF91CF911F91D3
:101BE0000F910895AF92BF92CF92DF92EF92FF9242
:101BF0000F931F93CF93DF9300D00F92CDB7DEB733
:101C0000182FF62E042FE22E90910C0390FF3AC06D
:101C1000E92FE695AE2FB0E0AB58BE4F8C91809384
:101C200061029E7F9230E1F59E012F5F3F4F812F31
:101C30000E945F0C4B8169818A810E945C0D8091BA
:101C40000D03811308C080910E038F1104C0809191
:101C50000F03801729F080916302826080936302F2
:101C600010930D03F0920E0300930F03EE2051F03A
:101C700060910C0370910D0380910E0390910F03FE
:101C80000E94800C0F900F900F90DF91CF911F91C9
:101C90000F91FF90EF90DF90CF90BF90AF9008959D
:101CA000823019F400910F03CACF863019F41091D5
:101CB0000D03C5CF8930D9F3893109F6E9518E2F4B
:101CC0008170D82EE695F0E0EF53F74FA590B490D1
:101CD000C12CBB2460911B01C61618F00E94FE0C9B
:101CE000AECF2C2D30E0A29EC001A39E900DB29EDF
:101CF000900D112470E00E948931812FD11013C002
:101D0000860F40911901420F532F511D9A01220F46
:101D1000331F240F351F2F5E3C4F402F6F2D0E9425
:101D20005F0CC394D7CF861BECCFECE0F3E091813E
:101D3000282F4381628188E0890F0C94F20D81E0A5
:101D40000C94950EECE0F3E09181282F43816281A1
:101D500088EF890F0C94F20D81E00C94A20EECE058
:101D6000F3E0628121E1620F08F46FEF282F4381D5
:101D700081810C94F20D81E00C94AF0EECE0F3E065
:101D8000628121E1621B08F460E0282F4381818198
:101D90000C94F20D81E00C94BE0EECE0F3E0438174
:101DA00021E1420F08F44FEF282F628181810C94CA
:101DB000F20D81E00C94CD0EECE0F3E0438121E1E3
:101DC000421B08F440E0282F628181810C94F20DBF
:101DD00081E00C94DC0E20E00C94F20DEF92FF9267
:101DE0001F93CF93DF93EC0110E0EE24EA94F12CE3
:101DF00060911B01161770F00E94FE0C9A818C8175
:101E000090FF27C08F5F8C83DF91CF911F91FF9050
:101E1000EF90089520911901422F410F5527551F2A
:101E2000CA019A01220F331F280F391F2F5E3C4F22
:101E300070E0C7010E949D31962F8C8140910F0365
:101E400060910E03199F800D11240E945F0C1F5F8B
:101E5000CFCF8150D8CF9F92AF92BF92CF92DF92D7
:101E6000EF92FF920F931F93CF93DF93EC018A8140
:101E7000BB24BA9480FD02C0BB24B3948C81811131
:101E80000AC081E0B81227C080911B018150809365
:101E9000060281E08C83A12C80911B01A816F0F032
:101EA0000E94FE0C8091060291E0B9125DC0811182
:101EB00056C080911B018150809306021C82DF91E5
:101EC000CF911F910F91FF90EF90DF90CF90BF9037
:101ED000AF909F90089510920602DBCF00911901F8
:101EE000CA2CD12C0C0D1D2D111DC801880F991F56
:101EF000080F191F0F5E1C4FF80111821082128209
:101F000034E0E32EF12C912C80910602890D813171
:101F100004F18F70082E000C990BC816D90691F4A5
:101F200080910F038E9DA0018F9D500D112455951A
:101F3000479555954795980160910E0380910D0343
:101F40000E945F0C9B0CF1E0EF1AF108E9F6A394F4
:101F5000A3CF87FFDFCF90911B01890FDBCF81508B
:101F600080930602BC82ABCF90E0019660911B018A
:101F700070E00E949D31809306028C83A0CFEF9287
:101F8000FF920F931F93CF93DF93EC018C8181110C
:101F900009C081E08C831092050292E090931601B3
:101FA000809315018091190190911A0123E0829F7D
:101FB000F0011124EF5EFC4F891768F110E003E097
:101FC00060911B01161768F10E94FE0C80911501AB
:101FD00020910502280F2093050290911601980F79
:101FE00090931601191654F4022E000C330B4091F5
:101FF0001B014150550B2417350734F08195809310
:102000001501813009F41C82DF91CF911F910F914E
:10201000FF90EF9008951182108212828F5F3396A5
:10202000CBCFE12EF12C70E0C7010E949D312091B1
:102030001901820F482F50E020910502022E000C5A
:10204000330BE216F306BCF020911601022E000CB1
:10205000330B2E153F057CF0809F900111242F5EDD
:102060003C4F40910F0360910E0380910D030E943D
:102070005F0C1F5FA5CFFA01EE0FFF1FE40FF51FE6
:10208000EF5EFC4F118210821282F3CF0F931F93E9
:10209000CF93DF938C01FC0184819581019681703F
:1020A000992795838483C0E0D5E580911B01C817EB
:1020B00030F0DF91CF911F910F910C94FE0C209185
:1020C0001901422F4C0F5527551FCA019A01220FA3
:1020D000331F280F391F2F5E3C4F8C2F8695F80138
:1020E00044815581840F952F911D817040910F037C
:1020F00060910E038D9F802D11240E945F0CCF5F95
:10210000D4CF0F931F93CF93DF93EC0110E000E047
:1021100090911B019017110609F06CF40E94FE0CBF
:102120008C8190E00196817099278C83DF91CF910B
:102130001F910F91089520911901A801420F511D7F
:102140009A01220F331F240F351F2F5E3C4F4C8105
:1021500060910E0380910D0396959017110651F032
:102160004CF0442349F040910F030E945F0C0F5F35
:102170001F4FCECF4423B9F340E0F7CF8F929F9209
:10218000AF92BF92CF92DF92EF92FF920F931F9385
:10219000CF93DF93FC01B280948081E0848300E0E0
:1021A00015E05BE4A52E88248394EE24EA94F12CB8
:1021B0007BE4C72ED12C80911B01081770F0DF91B2
:1021C000CF911F910F91FF90EF90DF90CF90BF9034
:1021D000AF909F908F900C94FE0CC02FD0E01C9F6E
:1021E000F0011D9FF00D1124E65FFD4F91101CC002
:1021F0001382128220911901CE01820F911D9C0140
:10220000220F331F280F391F2F5E3C4F1C9FF001F8
:102210001D9FF00D1124E65FFD4F42816181808199
:102220000E945F0C0F5FC7CF2381222379F12150D9
:10223000238334818A2D821B311101C0822F1C9F80
:10224000F0011D9FF00D1124E65FFD4F90910F03EB
:10225000899FC0011124B6010E9489316283211136
:1022600004C0332311F01482A38222E02B1510F254
:102270001C9FF0011D9FF00D1124E65FFD4F809122
:102280000D03808380910E038183B4CF0E940A32B4
:10229000823091400CF0AECF82E08B1530F50E9479
:1022A0000A32B7010E949D311C9FF0011D9FF00D65
:1022B0001124E65FFD4F808322E02B15C8F40E94B5
:1022C0000A3220910E032695622F70E00E949D3104
:1022D000280F1C9FF0011D9FF00D1124E65FFD4F9C
:1022E00021831282A382848285CF80910D03DCCF6B
:1022F00020910E03EECF8091630208951092630245
:10230000089525E0ECE0F3E0DC0101900D922A95C0
:10231000E1F7209161023091620240916302FC0179
:102320002583368347830895E1E6F2E011828281B6
:10233000846082830895ECE0F3E080818E7F808367
:102340000E949411E1E6F2E08281816082832FEFA6
:1023500080E792E0215080409040E1F700C000000B
:102360000C94FE0CECE0F3E080818E7F8083608132
:102370007181828193810E94800C0E949411E1E618
:10238000F2E08281816082832FEF80E792E021502A
:1023900080409040E1F700C000000C94FE0C60917A
:1023A0000C03669570E04BE050E08CE191E00E94F8
:1023B0001A32892B19F481E0809362020E94A728C7
:1023C00090935B0280935A028091630284608093B1
:1023D0006302089590910C0390FF3AC091708111AF
:1023E0002DC0926090930C03809163028160809372
:1023F0006302662351F060910C0370910D0380918C
:102400000E0390910F030E94800C60910C0366955F
:1024100070E04BE050E08CE191E00E941A32892B91
:10242000A1F00E94941181E080935D0240910F031E
:1024300060910E0380910D030C94EB0E8B3210F023
:102440009465D0CF880F982BCDCF0E94CF11EBCFC2
:102450000895682F90910C03969581E0890F8B3237
:1024600008F081E00C94EA1181E00C942912682FA5
:1024700090910C0396958FEF890F09F48AE20C94E2
:10248000EA1181E00C94371261E00C94EA11ECE05F
:10249000F3E080818160808386950C944412809162
:1024A0000C0380FD0C94B2110C94471260E00C9464
:1024B000EA1180916002811133C00E942C278111A2
:1024C00004C00E94C9270E949C0C0E947C0C60934F
:1024D0000C0370930D0380930E0390930F03809170
:1024E00063028360809363026E7F61F40E949C0CA0
:1024F0000E947C0C60930C0370930D0380930E0379
:1025000090930F030E946D0C0E94941180910C0314
:1025100080FF03C086950E94561281E0809360027E
:102520000895ECE0F3E080818160808386950C94CF
:1025300056121F93CF93DF93EC01162F8F8180FFEC
:102540000CC0888180FF24C080910C03816080933F
:102550000C03888186950E94EA118F8181FF06C055
:10256000212F4B816A8189810E94F20D8F8182FF28
:1025700005C08E81882379F00E94CF118F8183FF5F
:1025800003C081E080935D02DF91CF911F91089598
:102590000E949B11E2CF0E949411F0CFEF92FF9224
:1025A0000F931F93CF93DF9380916202882309F4E6
:1025B00068C080916102E0910C03E695E81BE0930E
:1025C0005C02823009F064C0F0E0E354F84FE4911B
:1025D000CE2FD0E00FE81DE080915D02882389F0C6
:1025E00010925D020E94A7289E0120953095820FCF
:1025F000931F90935B0280935A0210925F02109295
:102600005E0280915A0290915B020E94BF288C1753
:102610009D07B8F1809109028823B1F01092090258
:1026200080910702909108020E94BF28803395474D
:1026300058F00E94A7289093080280930702809187
:102640006302886080936302E0905E02F0905F0214
:10265000E0915A02F0915B02CE0FDF1FD0935B0234
:10266000C0935A028AE592E0F801099580915E02D2
:1026700090915F02892B29F4EF2819F081E0809373
:102680000902DF91CF911F910F91FF90EF90089574
:10269000863049F4F0E0E654F84FE491CE2FD0E0D4
:1026A00003EA1DE099CF893051F4E695F0E0E95452
:1026B000F84FE491CE2FD0E00EEE1EE08DCF8F309C
:1026C00051F4E695F0E0EC54F84FE491CE2FD0E0D1
:1026D0000BE21FE081CF853149F4F0E0EF54F84F71
:1026E000E491CE2FD0E00FEB1FE076CFC8EED3E021
:1026F00006E410E1883109F46FCF833239F4EFEA50
:10270000F7E0C591D49103EB1DE066CFC4EFD1E0B3
:1027100001E810E1843209F45FCFC0EDD7E009E5AC
:102720001CE0853209F058CF8E2F63E00E947D3186
:10273000E92FF0E0E455F84FE491CE2FD0E00EEB16
:1027400010E14ACFFA01811101C0FB010994CF9336
:10275000DF93C82FD62F0E94B30C8C1740F00E9435
:10276000B30C8D1720F4DF91CF910C9434128C2F81
:10277000DF91CF910C9444121F93CF93DF93EC0120
:10278000FB011281111110C00E9477268272FE0196
:10279000E25CFC45E431F10508F05BC0EC52FD4C15
:1027A0000C94B1310E944F12812FDF91CF911F9174
:1027B000089541E452E164E372E10E94A213F4CF70
:1027C00044E352E161E472E1F8CF4CEA5EE06FE984
:1027D0007EE0F3CF4FE95EE06CEA7EE0EECF4AECBC
:1027E0005EE06BEB7EE0E9CF4BEB5EE06AEC7EE017
:1027F000E4CF48EE5EE069ED7EE0DFCF49ED5EE0DC
:1028000068EE7EE0DACF4CEC5CE06BEB7CE0D5CFA1
:102810004BEB5CE06CEC7CE0D0CF81E00E9444129A
:10282000C3CF65E082E00E94A713BECF68E086E0D8
:10283000FACF6EE089E0F7CF64E18FE0F4CF67E193
:1028400085E1F1CF88E1EACF62E289E1ECCF83E272
:10285000E5CF11E0A9CF2AB1342F3F70A1E0B0E05D
:1028600001C0AA0F3A95EAF72A2B2AB942954F7070
:10287000E42FF0E022A14A2F4095422332A1A32B5E
:102880005FB7F8949B01220F331F260F371F280FC5
:10289000391F2817390741F45FBF87EC90E0019793
:1028A000F1F700C000000895FC016191CF0178E0CC
:1028B000ABB9000000C067FF4BB9660F000000C055
:1028C00000C000C04BB900C07A9591F7E2CF43E950
:1028D0000C942B140C94DA0580910401811106C02C
:1028E00080E38093280182E98093270120912801C9
:1028F000A22FA295AF70B0E091963C9191972F7066
:1029000081E090E0BC01022E01C0660F0A94EAF754
:10291000462F4095432391964C93919792963C91E4
:102920009297362B92963C93929740912701E42FF1
:10293000E295EF70F0E031A14F70042E01C0880FD6
:102940000A94EAF7982F9095932391A392A1892B4B
:1029500082A390968C9190E002C0959587952A95D8
:10296000E2F7817020A130E002C0359527954A95A5
:10297000E2F792E020FF90E0892B8093690290912A
:10298000040181E0982790936502891B809364027B
:102990000895CF93E0916902EE0FEE0F2091280188
:1029A000A22FA295AF70B0E090968C9190E02F701E
:1029B00002C0959587952A95E2F7817099274091F5
:1029C0002701A42FA295AF70B0E090962C9130E033
:1029D0004F7002C0359527954A95E2F7A9014170DD
:1029E000552720FF02C042E050E0842BE82BE09303
:1029F0006902C0916502EF70F0E0E056FE4F808101
:102A000090916802890F8093680284306CF0EC2FFB
:102A10000C2E000CFF0BEA59FD4F80818F5F8083E5
:102A200060E08C2F0E946A14809168028D3F6CF4E4
:102A3000EC2F0C2E000CFF0BEA59FD4F80818150CA
:102A4000808361E08C2F0E946A14809168028378F1
:102A500087FF03C081508C6F8F5F80936802CF9196
:102A60000895E0916502F0E0EA59FD4F2081FC01F4
:102A700020830895FF920F931F93CF93DF93D091FC
:102A800064020D2F10E00A591D4FFC01C081F801AE
:102A90008081C81BFC2E1F1464F08C2FC7FD80E0C2
:102AA000C81BC11110C0DF91CF911F910F91FF90F2
:102AB0000895FA94F80180818F5F808360E08D2F04
:102AC0000E946A14E8CFCF5FF80180818150808333
:102AD00061E08D2F0E946A14E4CF82E290E00E94B0
:102AE0002732813289F483E290E00E9427328330DA
:102AF00059F484E290E00E94273291E0803209F09C
:102B000090E0892F8170089580E0FCCFCF93C82F8B
:102B10006FEF811161E282E290E00E943B326FEF41
:102B2000C11163E083E290E00E943B326FEFC1117C
:102B300060E284E290E0CF910C943B3280E00E940E
:102B400086150C942627089585E290E00E9427328E
:102B5000682F70E090E080E0089585E290E00C94AA
:102B60003B320E94A3150E946D1581110CC060E0DC
:102B700070E0CB010E94AD150E9467170E945318A8
:102B800081E00C9486150895CF93FB01C281CC237C
:102B900009F19C0122513F452031310520F5825138
:102BA0000E946318C0E08C2FCF91089581E00E94AD
:102BB000EF2443E062E081E00E943D07F3CF81E033
:102BC0000E94102543E062E081E00E943D07EBCFC8
:102BD00082E0F6CF8031FFE59F0789F381319F4581
:102BE000B9F3C1E0E0CF8031EFE59E07F9F2813122
:102BF0009F45C9F682E0DBCF2FEFFC0120830895CB
:102C0000CF93DF93EC0188818138A9F028F48038D4
:102C100071F0DF91CF910895823881F08338C9F740
:102C20000E94F20C89830E94F50C8A83F2CF0E94E5
:102C3000F80C8983EECF0E94B30CFBCF0E94DD0C11
:102C4000F8CFCF93DF93EC0188818138E1F028F44D
:102C5000803869F0DF91CF910895823811F183387F
:102C6000C9F70E94F80C482F6A81898108C0D98170
:102C70000E94F50CC82F0E94F20C4D2F6C2FDF9193
:102C8000CF910C94EB0E89810E945612898181119B
:102C900004C0DF91CF910C949B11DF91CF910C94E4
:102CA00091128981DF91CF910C94EF0CEF92FF92FA
:102CB0000F931F93CF93DF93EC01062FDC01ED916F
:102CC000CD01E150E33108F0BFC0F0E0E851FD4C28
:102CD0000C94B131198289E08A83602FCE01DF9193
:102CE000CF911F910F91FF90EF900C94A12A8981B1
:102CF000823069F0833071F08130D9F40E94B328BA
:102D00000E94B7316A837B838C839D83E6CF0E94C8
:102D1000A415F6CF7E01B2E0EB0EF11C10E0812F7E
:102D20000E94BE09F70181937F011F5F1830B9F738
:102D3000D4CF602FCE010E94FC15CFCF8981823085
:102D4000C1F76A817B818C819D810E94B7310E948D
:102D5000AD15C3CF4B816A8189810E9439179827AD
:102D6000892798279D838C83B8CF2C813D8132277A
:102D7000232732274B816A8189810E945217ADCF68
:102D80000E946717AACF0E942116A7CF0E940016A3
:102D9000A4CF0E94920CA1CF0E94FC1789839DCFE3
:102DA0000E94FE179827892798279A83898395CFB1
:102DB0006B8170E089819A81AE014C5F5F4F9827EB
:102DC000892798270E94011888CF6B8170E089813C
:102DD0009A81AE014C5F5F4F9827892798270E9400
:102DE00028187BCF0E94531878CF0E942717D6CF80
:102DF0006B8170E089819A81AE014C5F5F4F9827AB
:102E0000892798270E949F1768CF6B8170E089817E
:102E10009A81AE014C5F5F4F9827892798270E94BF
:102E2000C5175BCF0E949E1558CFCE010E94A12AE4
:102E3000FFEF21EE84E0F15020408040E1F700C038
:102E400000000E94F22849CF8FEF888346CF84E0AC
:102E5000089550E0440F551F9CE0699F400D511D9F
:102E6000112490E6899F400D511D1124CA018696B8
:102E700008950F931F93CF93DF930E9429178C011E
:102E80000E942732C82FD0E0DC2FCC27C801019642
:102E90000E9427329E01282BC901DF91CF911F91FB
:102EA0000F9108950F931F93CF93DF93122F032F4A
:102EB0000E942917EC01602F0E943B32612FCE0146
:102EC0000196DF91CF911F910F910C943B32AF92FD
:102ED000BF92CF92DF92EF92FF921F93CF93DF9337
:102EE0008CEAC82E80E0D82ED0E07601C0E014C075
:102EF000F50125913491412F6C2F8D2F0E9452178F
:102F000082E0A80EB11C1F5F163091F78CE0E80E2E
:102F1000F11CCF5FC83019F0570110E0E9CFDF5F37
:102F200080E6C80ED11CD43001F7DF91CF911F91FC
:102F3000FF90EF90DF90CF90BF90AF900895EF9209
:102F4000FF920F931F93CF93DF93EC018A017C01D3
:102F5000E60EF71ECE018696CE15DF0539F4DF9119
:102F6000CF911F910F91FF90EF900895C03821E00D
:102F7000D20740F40E942732F80180830F5F1F4F71
:102F80002196E8CFF8011082F9CFCF92DF92EF922D
:102F9000FF920F931F93CF93DF937C016A018C0103
:102FA000060F171FEC01CE018696C017D10749F412
:102FB000DF91CF911F910F91FF90EF90DF90CF9015
:102FC0000895C03821E0D20740F4FE01EE19FF0950
:102FD000EC0DFD1D60810E943B322196E4CF462F0F
:102FE000843038F4783028F4663018F4672F0C9465
:102FF000391790E080E0089580E108958AE592E035
:103000000895EF92FF920F931F93CF93DF93EC01FC
:103010008A017C01E60EF71ECE018A559E4FCE1521
:10302000DF0539F4DF91CF911F910F91FF90EF9061
:103030000895CA3522E0D20740F40E942732F801F1
:1030400080830F5F1F4F2196E7CFF8011082F9CFE1
:10305000CF92DF92EF92FF920F931F93CF93DF9364
:103060007C016A018C01060F171FEC01CE018A5505
:103070009E4FC017D10749F4DF91CF911F910F9157
:10308000FF90EF90DF90CF900895CA3522E0D207ED
:1030900040F4FE01EE19FF09EC0DFD1D60810E9458
:1030A0003B322196E3CFCF93DF93C6EAD1E060E0D5
:1030B000CE010E943B322196C11584E0D807B9F7B2
:1030C000DF91CF910895DF92EF92FF920F931F93BC
:1030D000CF93DF9300D000D0CDB7DEB7F82E8FE0CE
:1030E0008F1540F08FEF93E00E94273206EA11E03F
:1030F0008823C1F00F900F900F900F90DF91CF9128
:103100001F910F91FF90EF90DF900895011584E0DB
:10311000180781F3C8010E942732811101C0FA9477
:103120000F5F1F4FF110F2CF19821A821B821C828F
:10313000DD24D39478018FEFE81AF80AC8010E94C1
:10314000273289831A828823A9F29FEF980F933040
:1031500078F48A83D9820E5F1F4FC7010E942732FD
:103160008B83882339F2CE0101960E94E606E2CFD6
:103170008701F9CF0F931F93CF93DF93C62FD42FDF
:10318000022FFC0182818823C9F060936C020E94A7
:10319000A72890936B0280936A0280E28C0F88309C
:1031A00008F050C0C77081E001C0880FCA95EAF7E7
:1031B000DF91CF911F910F910C949A1E10916C0288
:1031C000161335C080916A0290916B020E94BF284D
:1031D000883C910560F5C0E2CD0F1D17B9F080E283
:1031E000810F883040F4177081E001C0880F1A9574
:1031F000EAF70E94A11EC83048F481E09D2F977025
:1032000001C0880F9A95EAF70E949A1E802F0E94AB
:10321000871EC830B8F4D77081E001C0880FDA95F6
:10322000EAF7DF91CF911F910F910C94A11E80E2DC
:103230008C0F883038F4C77081E001C0880FCA95C0
:10324000EAF7EFCFDF91CF911F910F9108959C0185
:10325000CB01233F4CE5340731F190F4283DFCE5E8
:103260003F07E9F0293D4CE5340769F1273D3C452E
:1032700079F426E241EE61EE0E94BA1880E00895EA
:10328000253FFCE53F07B9F090F0263F3C45B9F0FB
:10329000FC0182818823D1F010926C02089527E20C
:1032A00045EE65EEE9CF26E241EE60EEE5CF27E29E
:1032B00045EE64EEE1CF26E241EE62EEDDCF27E29D
:1032C00045EE66EED9CF28E241E0EBCF81E00895EC
:1032D000CF93DF93EC01FB018281882309F419C1AC
:1032E000C230FCE5DF07C0F1C6319CE5D90730F0FC
:1032F0009E012A5F3C452930310570F50E943F2729
:103300009093460380934503C031ECE5DE0709F452
:10331000CFC008F05BC0C8308CE5D80709F4B6C050
:1033200088F5C430ECE5DE0709F4A8C0C0F4C2306B
:103330008CE5D80709F49CC0809145038260C330B6
:10334000DC4509F498C080914503909146030E94A2
:103350004D270E94F72080E0DF91CF910895809162
:1033600045038061C630ECE5DE0709F484C0809136
:1033700045038860C730DC4508F47DC08091450373
:10338000806279C0CC308CE5D80709F489C070F42C
:10339000809145038C60CA30ECE5DE0709F46BC010
:1033A00008F478C0809145038E7F65C0CE308CE5EF
:1033B000D80709F479C0809145038B7FCF30DC4575
:1033C00008F459C0809145038F7E55C0CB3FECE592
:1033D000DE0709F457C030F5C3318CE5D80709F48E
:1033E0006FC078F4C131ECE5DE0709F465C0C23185
:1033F000DC4509F0A8CF0E94F720809145038F7724
:103400003AC0C5318CE5D80709F462C008F476C02B
:10341000809146038160CA3FDC4509F094CF8093D8
:10342000460391CFCF3FFCE5DF0709F44DC088F498
:10343000809146038D7FCD3F9CE5D90781F3809134
:1034400046038E7FCE3FDC4550F380914603836078
:10345000E6CFC130FDE5DF0709F459C008F444C0E8
:1034600080E0C230DD4509F06ECF0E94CB276BCFE4
:103470008091450381608093450365CF809145032A
:103480008460F9CF809146038260C9CF8091450363
:103490008064F1CF0E94F720809145038068EBCFD4
:1034A000809145038D7FE7CF80914503877FE3CFF0
:1034B000809145038F7DDFCF809145038F7BDBCFEC
:1034C00080914503837FD7CF809146038C7FA7CF20
:1034D0008091450382FB992790F921E0922790FB88
:1034E00082F990FB83F9C7CF80914603982F90957E
:1034F00091708E7F892B90FB81F991CF0E94F720EC
:1035000090914503892F97FB87F98058B4CF81E0CC
:10351000ACCF81E021CFCF93DF93EB0186319C4587
:1035200011F50E9477269A81992399F08A7A91E081
:1035300009F490E090936D02811109C089E20E9424
:1035400052260E94C32680E0DF91CF91089585E343
:10355000F6CF80916D02811104C089E20E94592644
:10356000F0CF85E3FBCF81E0EFCF8EE1489B02C037
:103570008150E1F7489BFECF0895589880E28A95E4
:10358000F1F7589A0895FC013BE03A95F1F720E0F5
:1035900090E080E031E040E14A95F1F7880F489BE8
:1035A00002C08160232742E04A95F1F7000040E124
:1035B0004A95F1F79F5F6913EECF90E19A95F1F785
:1035C00099B132E03A95F1F7000040E14A95F1F700
:1035D000917092272081920F90830895EF92FF922D
:1035E0000F931F93CF93DF930F92CDB7DEB719825E
:1035F0008C017C01E60EF11C0E151F0561F481E0C3
:103600009981911180E00F90DF91CF911F910F91DF
:10361000FF90EF9008950E94B51A68E0CE010196E0
:103620000E94C31AF80181938F01E6CF9093700234
:1036300080936F0260936E02509A589A0895909307
:10364000700280936F0260936E025098589AE89AC5
:10365000E9E6F0E080818C7F808308956150770BEC
:1036600091E001C0990F6A95EAF720E031E09111ED
:1036700008C0222391F0589A80E28A95F1F7589871
:103680000895492F482339F0589A232740E24A9554
:10369000F1F79695ECCF5898F9CF5898EDCFFF9267
:1036A0000F931F93CF93DF93EC018C01060F111D35
:1036B000C017D10731F4DF91CF911F910F91FF9087
:1036C0000895F9900E94BD1A68E08F2D0E942E1B6C
:1036D000EFCF1F920F920FB60F9211240F931F93EB
:1036E0002F933F934F935F936F937F938F939F930A
:1036F000AF93BF93EF93FF93CF93DF930F92CDB729
:10370000DEB719820E94B51A67E0CE0101960E94C9
:10371000C31A082F069506950695982F92959570D1
:10372000202F2570920F292F2370969596958770DC
:10373000920F891344C08981811141C080916E022A
:103740008017E8F120E12A95F1F7589A509A82E023
:103750008A95F1F700C0A8E00A9FC00111240091EA
:103760006F0210917002080F191F5898F8016581B7
:10377000662321F0868197810E944F1B0E94BD1A0B
:10378000F0E1FA95F1F758985098589A20E12A9567
:10379000F1F7D80112966C911297662331F11396C6
:1037A0008D919C910E94EE1AD801ED91FC91882395
:1037B00011F088E001C082E080830E94B51A0F906A
:1037C000DF91CF91FF91EF91BF91AF919F918F9139
:1037D0007F916F915F914F913F912F911F910F9129
:1037E0000F900FBE0F901F901895ED91FC91E1CFB7
:1037F0000F931F93CF93DF9320916E022817190622
:103800000CF471C08C0193E0000F111F9A95E1F741
:10381000C0916F02D0917002C00FD11FF894509ADE
:10382000589825E02A95F1F70000982F9695957005
:103830008570980F892F837096959695980F092B10
:103840000E94BD1A00C067E0802F0E942E1B80E1FD
:103850008A95F1F75098589A489B17C087E090E0F6
:10386000489915C06D81662321F18E819F810E9448
:10387000EE1A81111EC0509A589AE881F98182E0AF
:103880008083789482E090E00DC000C0E5CF01977E
:1038900071F4509A589AE881F98181E08083789494
:1038A00081E090E0DF91CF911F910F91089500C0CA
:1038B000D7CF0E94B51A20E22A95F1F75898509A6E
:1038C00080E18A95F1F76A81662321F08B819C81E2
:1038D0000E944F1B0E94BD1AE881F98110827894E2
:1038E00090E080E0DFCF84E090E0DCCF9093760240
:1038F000809375020895E0917502F09176023097F9
:1039000021F00190F081E02D099480E00895E0918C
:103910007502F0917602309721F00280F381E02D5C
:103920000994089520917302309174022817390781
:1039300071F09093740280937302E0917502F0919C
:103940007602309721F00680F781E02D09940895E2
:1039500020917102309172022817390771F090930B
:10396000720280937102E0917502F09176023097B5
:1039700021F00084F185E02D0994089585B78068D1
:1039800085BF85B7806885BF0895089508950C9414
:10399000C51C08950C94C91C0E94BE1C0E94C61C24
:1039A0000C94C71C0C94320B0E949E280E94CA09DA
:1039B0000E94B1150E942C290E9459120C94CA1C15
:1039C000AF92BF92CF92DF92EF92FF920F931F932D
:1039D000CF93DF93CDB7DEB72A970FB6F894DEBF4B
:1039E0000FBECDBF0E944E0A0E94D21C882309F44C
:1039F0005FC088E7A82E82E0B82E10E000E0C02E5D
:103A0000802F0E94BE09E82EF501D1905F01D816E3
:103A100009F448C08091EC0281FD0E94C40980E055
:103A2000FF24F394DE249D2D9F21B9F18E83CF8254
:103A3000EF2081E009F480E088870E94A728816058
:103A4000782F9A8789874E815F8168858A850E9451
:103A50007A1DF801E858FD4F8081F826F0820E9417
:103A6000CE120E947B1C90917702891791F10E94DF
:103A70007B1C809377022A960FB6F894DEBF0FBEA8
:103A8000CDBFDF91CF911F910F91FF90EF90DF900D
:103A9000CF90BF90AF900C9466078F5FFF0C86307D
:103AA00009F0C1CF0F5F1F4F0830110509F0A7CFF4
:103AB0008FEF89838A831B820E94A7288160782FD9
:103AC0009D838C8349815A816B818D810E947A1DEF
:103AD000C6CF2A960FB6F894DEBF0FBECDBFDF91DA
:103AE000CF911F910F91FF90EF90DF90CF90BF90FB
:103AF000AF900895CF93DF93CDB7DEB72B970FB676
:103B0000F894DEBF0FBECDBF4F83588769877A8791
:103B10008B871E821D8285E0FE013796DE0111969D
:103B200001900D928A95E1F749815A816B817C81E0
:103B30008D819E812B960FB6F894DEBF0FBECDBF50
:103B4000DF91CF910C946D23FC01808191810C94C5
:103B50002426CF93C82F882309F488C08238C1F463
:103B60000E947B1C81FD82C089E30E9452260E9434
:103B7000C3262FEF81EE94E0215080409040E1F782
:103B800000C0000089E30E945926CF910C94C326FF
:103B90008338A1F40E947B1C80FD68C083E50E94ED
:103BA00052260E94C3262FEF81EE94E021508040E0
:103BB0009040E1F700C0000083E5E5CF8438A1F430
:103BC0000E947B1C82FD52C087E40E9452260E9404
:103BD000C3262FEF81EE94E0215080409040E1F722
:103BE00000C0000087E4CFCF8CEF8C0F813AB8F48F
:103BF0008C2F0E94EB29811139C06C2F80912901F3
:103C000090912A010E94E227882329F08C2F0E949C
:103C100059260E94C3268C2F0E945226B6CF80E2DE
:103C20008C0F883048F4C77081E001C0880FCA95B6
:103C3000EAF70E947A26A9CFEBE5EC0FE33040F4D7
:103C4000F0E0E252FE4F808190E0CF910C94921C04
:103C5000C85AC73158F4EC2FF0E0EE0FFF1FE055C3
:103C6000FE4F80819181CF910C94A81CCF91089533
:103C7000882309F44BC0823871F40E947B1C81FFB9
:103C800045C089E30E9452260E94C32689E30E9410
:103C900059260C94C326833859F40E947B1C80FF5C
:103CA00035C083E50E9452260E94C32683E5EFCFEC
:103CB000843859F40E947B1C82FF28C087E40E944C
:103CC00052260E94C32687E4E2CF9CEF980F913AD8
:103CD000F0F290E2980F983050F4877091E001C0B4
:103CE000990F8A95EAF7892F0E948026D2CF9BE50B
:103CF000980F933020F490E080E00C94921C885A46
:103D0000873120F490E080E00C94A81C0895CF93B4
:103D1000C82F0E94A91DC93349F42FEF87EE93E005
:103D2000215080409040E1F700C000008C2FCF91DF
:103D30000C94381E882321F00E947A260C94C32606
:103D40000895882321F00E9480260C94C3260895AC
:103D5000BF92CF92DF92EF92FF920F931F93CF9378
:103D6000DF936C01D62FC72FFC01058102950F70E0
:103D7000128111110E9497260E947026E82E882336
:103D800071F01123B1F080E28D0F883090F082E065
:103D90000E940E270E94702691E0E82EE926BC2E94
:103DA000B2949FE0B922EB2DF0E0E550FD4C0C946D
:103DB000B131E12CF4CF0C2F0F70C07F11F00295C0
:103DC000007F1123A9F0002359F080E28D0F883085
:103DD00010F0D11109C0802F0E947A260E94C326BC
:103DE0008D2F0E94A91D14C0802F0E948A26F6CF15
:103DF0008D2F0E94381E002359F080E28D0F8830ED
:103E000010F0D1112CC0802F0E9480260E94C32662
:103E10002B2D2850330B2430310520F40E947B1CBD
:103E20000E946607EE2009F493C10E946C2680FD73
:103E30008FC1F60112820E9466260E94EF24C601FD
:103E40000E94C9200E946626DF91CF911F910F9199
:103E5000FF90EF90DF90CF90BF900C941025802FB3
:103E60000E949026D3CFFC2FFF70FF2EC07FC03260
:103E700019F0F29480EFF822DD2369F0D13049F196
:103E8000112391F1002351F1F601858180FFA8CF24
:103E90008F70858323C0112381F0011106C00E9419
:103EA000AA268F290E949A1EB3CF0130C1F70E9423
:103EB000AA268F290E94B026ABCF011106C00E940E
:103EC000B9268F2D0E94A11EA3CF013009F4A0CFE7
:103ED000F6CF112329F0063008F09ACF8F2DE2CFCC
:103EE000053008F095CFEDCF002359F3D93349F4CD
:103EF000FFEF27EE33E0F15020403040E1F700C003
:103F000000008D2F0E94381E83CF8C2F86958695BA
:103F1000837069F0813009F07BCF8D2F9C2F9370D7
:103F2000111102C090E080E00E94A81C71CF8D2F7B
:103F30009C2F9370111102C090E080E00E94921CAF
:103F400067CF8C2F837009F041C0111161CF4D2FC5
:103F5000429546954770440F440F0D2F0F7010E0A7
:103F600030E020E0042E04C0000F111F221F331F79
:103F70000A94D2F760E070E0CB01D4FF0FC06FE08D
:103F800070E080E090E004C0660F771F881F991FE3
:103F90004A95D2F76095709580959095C695C6958F
:103FA000C370602B712B822B932BC23049F058F4D5
:103FB000C13019F00E94A3242BCF0E94912428CF56
:103FC0000E94B52425CF0E948F2422CF86951123ED
:103FD00011F08C2F8170882309F41ACF4D2F429550
:103FE00046954770440F440F0D2F0F7010E030E0DE
:103FF00020E0042E04C0000F111F221F331F0A945B
:10400000D2F760E070E0CB01D4FF0FC06FE070E04A
:1040100080E090E004C0660F771F881F991F4A95C3
:10402000D2F76095709580959095C695C695C370AA
:10403000602B712B822B932BC23049F058F4C13086
:1040400019F00E946625E4CE0E945425E1CE0E941C
:104050007825DECE0E94C924DBCECF70112329F053
:104060008C2F0E94EF248D2F1DCF8D2F0E94A11E1B
:104070008C2F0E941025CCCED23F89F160F4D03F26
:10408000C9F0D13F29F1112309F442C00111A8CE92
:104090008C2F8F7121C0D33F39F1D43FA1F7112369
:1040A00069F1CF718C2F0E94EF2463E08C2F0E9466
:1040B000F926AECE112341F0053008F0A9CE8C2FA1
:1040C0008F710E943325A4CE063008F0A1CEF7CF21
:1040D0008C2F8F71112369F20E94EF2499CE8C2FBF
:1040E0008F711123C9F3C5CF112329F08C2F8F7144
:1040F0000E94DA248DCE0E94D5248ACE81E00E94CF
:104100000E27023008F484CE82E00E940E2780CE73
:10411000002359F0D93309F0F4CE8FEF97EEE3E0A6
:1041200081509040E040E1F7EACE8C2F8F71A1CF13
:104130004C2F4F706D2FC6010E94C6070E940724A6
:1041400067CE4C2F4F706D2FC6010E94C90760CEFD
:10415000DF91CF911F910F91FF90EF90DF90CF9063
:10416000BF9008950F931F93CF93DF93EC01688165
:1041700079818A810E942E268C010E948A250E94C4
:104180008E24B801CE01DF91CF911F910F910C9435
:10419000A81ECF93DF93EC018B819C81892B29F0A2
:1041A0008881998189238F3F19F4DF91CF910895F8
:1041B000CE010E947E078823C1F3CE010E94B22067
:1041C000CE01DF91CF910C9425060E9497260E9484
:1041D000A7260E94C32690E080E00E94921C90E0F7
:1041E00080E00C94A81C0E9460260C94E5200E949C
:1041F00087260C94F320E92FE295EF70E250EE3021
:1042000070F4F0E0E55FFC4C0C94B131803F19F0A4
:1042100020F4883E20F481E00895843FE1F380E0BB
:104220000895883EC0F3813FD1F7F5CF93FB8827EF
:1042300080F908950E9424260C94FB20CF93DF93ED
:1042400000D000D00F92CDB7DEB70F900F900F9037
:104250000F900F90DF91CF910895CF93DF9300D00F
:1042600000D000D0CDB7DEB726960FB6F894DEBFEB
:104270000FBECDBFDF91CF9108951F93CF93DF93F2
:10428000C091810216E0809182028C1304C0DF91FC
:10429000CF911F910895D0E01C9FF0011D9FF00D5C
:1042A0001124ED57FD4F40815181628173818481DA
:1042B00095810E942D212196C770E5CF4091B302D0
:1042C0005091B4026091B5027091B6028091B7022C
:1042D0009091B8020C942D211F93CF93DF9380917E
:1042E000B802807FA9F48091B502882389F080917B
:1042F0008102C09182026091B3027091B402A091D8
:10430000B602B091B702D62FD72316E0C81304C067
:10431000DF91CF911F91089590E0109711F0DF3F4A
:1043200019F401968770F2CF189F9001199F300DF4
:104330001124F901ED57FD4F41814713F2CF408120
:104340004613EFCF42814111ECCF438154814A1B88
:104350005B0B483C510528F78091B8028F70806153
:104360008093B802F901E857FD4F80818F7080611A
:10437000808383EB92E00E94C920DF91CF911F914F
:104380000C943D21AF92BF92CF92DF92EF92FF92B9
:104390000F931F93CF93DF93CDB7DEB761970FB61F
:1043A000F894DEBF0FBECDBF8C0185E0F801DE01C1
:1043B0001D9601900D928A95E1F7F8014081518197
:1043C000E28083EBC82E82E0D82E6091B602709115
:1043D000B7026115710509F461C19091B302209192
:1043E000B402892F82238F3F09F458C1A380B4807F
:1043F000F090B502F501E61BF70BFF2009F4FCC0B5
:104400008091B802382F307FE83CF10508F0B2C047
:10441000311179C0FE2C251323C0941321C0E11063
:104420001FC08F7080618093B8020E945E21C60118
:104430000E94C9208091B802F80185838F2D619672
:104440000FB6F894DEBF0FBECDBFDF91CF911F91A5
:104450000F91FF90EF90DF90CF90BF90AF900895B5
:10446000AB2829F0842F85238F3F09F033C180E0EA
:10447000F82FF170DF2E80FF3CC0809181022091E7
:10448000820236E0821315C04D875E878D859E853A
:104490000E942426292F22952F702230F0F02430FC
:1044A00018F59F70F1F0F8019581907FD1F4D12C2F
:1044B0001EC090E0389FF001399FF00D1124ED5798
:1044C000FD4F6181651306C06081641303C0628182
:1044D0006E110FC001968770D5CF9F7011F08823A1
:1044E00031F3805E883018F3C8010E94C920FD2C8A
:1044F000A5CFEE2009F4A2CF8091B802816080930D
:10450000B802F12C9BCF251306C0941304C0F80108
:10451000EE2009F48DC04D875E878D859E850E94B3
:104520001A21882319F1EE2009F18091B802803216
:1045300070F02091B3023091B40238872F8319862E
:10454000BB86AA868C87CE0107960E94C92086E08A
:10455000F801A3EBB2E001900D928A95E1F70E9479
:104560006C210E945E21FF24F39468CFC8010E9451
:10457000C920F9CF311113C07A2DB98AA88A6E2DBE
:1045800089890E941E2183EB92E00E94C92086E067
:10459000F60111928A95E9F70E945E21B2CF2513A8
:1045A0000FC094130DC0E1100BC0F8018583C80142
:1045B0000E94C92086E0F60111928A95E9F73ECF64
:1045C0004D875E878D859E850E941A21882371F212
:1045D000EE2061F28091B802803208F4B8CF2091C9
:1045E000B3023091B4023A8329831B82BD82AC822C
:1045F0008E83CE010196A9CFE83CF10508F041C0B9
:10460000FE2CEE2009F4B2CF25132AC0941328C043
:104610008091B80280FD1BC0982F907FC1F0F801F7
:104620008583903F31F0982F907F905F8F70892B1A
:104630008583C8010E94C92086E0F801A3EBB2E09F
:1046400001900D928A95E1F70E945E21F7CE86E0F7
:10465000F801A3EBB2E001900D928A95E1F7EECE5E
:104660004D875E878D859E850E941A2181116FCFAF
:104670008091B80281608093B802C8010E94C9206D
:10468000DDCE7A2DB98AA88A6E2D89890E941E21D5
:1046900086E0F60111928A95E9F7D6CFEE2009F46B
:1046A00065CF4D875E878D859E850E941A21F82EE5
:1046B000882309F45BCF86E0F801A3EBB2E0019018
:1046C0000D928A95E1F783EB92E00E94A41D0E946F
:1046D0006C21BACF81E08E25CBCE1F93CF93DF9391
:1046E000CDB7DEB72C970FB6F894DEBF0FBECDBFA7
:1046F0004F83588769877A878B879C87CE01079677
:104700000E94C221882369F08A859B85892B39F014
:104710004F815885842F85238F3F09F071C016E0A3
:104720005FC086E0FE013796DE01119601900D9282
:104730008A95E1F78A859B85892B89F388859F81F6
:1047400089238F3F61F32091820230E0C9010196F5
:1047500087709927409181024817190671F40E94C9
:10476000F720109282021092810286E0E3EBF2E0E1
:10477000DF011D928A95E9F7D2CF96E0929FD00192
:10478000939FB00D1124AD57BD4FFE01319601909E
:104790000D929A95E1F7809382020E943D21BFCF4E
:1047A000819FC00111248D579D4F0E94C2218823F3
:1047B000E9F0E09181021E9FF0011124ED57FD4FB9
:1047C0004081518162817381848195810E942D2174
:1047D0008091810290E001968770992780938102F1
:1047E00080918102909182028913DACF2C960FB6C4
:1047F000F894DEBF0FBECDBFDF91CF911F9108951A
:1048000069857A858B859C850E942D2188CFEF92C2
:10481000FF920F931F93CF93DF938C01892B81F02D
:10482000F12CEE24E394E8012196F8018491843779
:1048300070F4843008F05FC08130B1F08230A1F1B3
:10484000DF91CF911F910F91FF90EF9008958537E1
:1048500009F44CC008F43DC09CE7980F903780F7EE
:104860008F770E94381E49C00E5F1F4FFE01849152
:1048700090E2980F983060F48770FE2D01C0FF0F12
:104880008A95EAF78F2F0E949A260E94C32602C0BB
:104890000E94A91D8F2D815030F2EFE9FFE0319782
:1048A000F1F700C00000F7CF0E5F1F4FFE018491AB
:1048B00090E2980F983050F48770FE2D01C0FF0FE2
:1048C0008A95EAF78F2F0E94A026DFCF0E94381E1C
:1048D000E1CF0E5F1F4FFE01C491C150D8F28FE9A6
:1048E0009FE00197F1F700C00000F7CF0E5F1F4F68
:1048F000FE01F490CFCF0E94A91D8E01CBCF089569
:104900000C947F240E9480246093DB027093DC026D
:104910008093DD029093DE020C94E52008950C94C0
:1049200082240F931F930091DB021091DC022091EF
:10493000DD023091DE02602B712B822B932B1F91B5
:104940000F910C9482240F931F930091DB0210911E
:10495000DC022091DD023091DE026023712382238C
:1049600093231F910F910C9482240F931F93009116
:10497000DB021091DC022091DD023091DE02602723
:104980007127822793271F910F910C9482240C94F6
:10499000D2050E94C7246093D7027093D8028093F7
:1049A000D9029093DA020C94E52060E070E0CB012C
:1049B0000C94C9240F931F9341E050E060E070E035
:1049C0008A019B0104C0000F111F221F331F8A950B
:1049D000D2F7C901B8011F910F910C94C9240F930C
:1049E0001F9341E050E060E070E004C0440F551FA9
:1049F000661F771F8A95D2F78091D7029091D802CF
:104A0000A091D902B091DA028A019B01082B192BDF
:104A10002A2B3B2BC901B8011F910F910C94C9247B
:104A20000F931F9341E050E060E070E004C0440F3A
:104A3000551F661F771F8A95D2F7CB01BA01609583
:104A40007095809590950091D7021091D802209191
:104A5000D9023091DA0260237123822393231F91BC
:104A60000F910C94C9240F931F9341E050E060E034
:104A700070E004C0440F551F661F771F8A95D2F758
:104A80008091D7029091D802A091D902B091DA0218
:104A90008A019B01082719272A273B27C901B8014A
:104AA0001F910F910C94C9240F931F930091D7026B
:104AB0001091D8022091D9023091DA02602B712B2B
:104AC000822B932B1F910F910C94C9240F931F934A
:104AD0000091D7021091D8022091D9023091DA02C8
:104AE00060237123822393231F910F910C94C92477
:104AF0000F931F930091D7021091D8022091D902F1
:104B00003091DA0260277127822793271F910F9136
:104B10000C94C9240895E92FEE0FE90FEE0F8E0FC4
:104B2000982F977041E001C0440F9A95EAF7869557
:104B30008695869595E0899FF0011124E754FD4FF5
:104B400030E020E070E05191DF011197CB01022E9F
:104B500002C0969587950A94E2F781708195852722
:104B6000842385278C932F5F3F4F2530310559F7DC
:104B70000895E92FEE0FE90FEE0F8E0F982F977023
:104B800086958695869525E0829FF0011124E7544D
:104B9000FD4F50E040E080E0219130E0092E02C05E
:104BA000369527950A94E2F721703327042E01C029
:104BB000220F0A94EAF7822B4F5F5F4F4530510571
:104BC00059F70895BF92CF92DF92EF92FF920F9321
:104BD0001F93CF93DF938C01C090D702D090D8025F
:104BE000E090D902F090DA028091DB029091DC0231
:104BF000A091DD02B091DE02C82AD92AEA2AFB2A56
:104C0000CFE1D0E0BC2ED701C6010C2E04C0B69572
:104C1000A795979587950A94D2F780FD0EC02197A6
:104C200088F7B12C8B2DDF91CF911F910F91FF90C1
:104C3000EF90DF90CF90BF900895B8018C2F0E9425
:104C4000D207019761F3EECFCF93DF93EC010E947F
:104C5000E225BE01DF91CF910C94D2071F93CF9331
:104C6000DF93EB0190918002992331F0CB01DF912A
:104C7000CF911F910C942426882379F0CB010E94B8
:104C8000E225182F682FCE010E948B25BE01812FAF
:104C9000DF91CF911F910C94D207CB010E94B925CF
:104CA000182FF4CF682F8091290190912A010C943C
:104CB0001828682F8091290190912A010C941A28B4
:104CC0008091290190912A010C941C288091DF0287
:104CD00085958595859508958091DF028770089563
:104CE0009091DF02977081E009F480E0089580914F
:104CF000EB0208959091EB02892B8093EB020895CB
:104D000080959091EB0298239093EB020895109276
:104D1000EB0208959091EA02892B8093EA020895AC
:104D200080959091EA0298239093EA020895109258
:104D3000EA0208959091E902892B8093E90208958F
:104D400080959091E90298239093E902089510923A
:104D5000E90208958091E002089508950C94AD262B
:104D60009091E002981721F08093E0020C94AE2617
:104D700008958091E002882329F01092E00280E0FB
:104D80000C94AE260895E0912901F0912A018091BA
:104D9000EB028083E0912901F0912A0180819091BA
:104DA000EA02892B8083E0912901F0912A01808118
:104DB0009091E902892B80839091E002992381F000
:104DC000E0912901F0912A018081892B80838091D3
:104DD000290190912A010E94D02781110E94B926B1
:104DE0008091290190912A010C94871C08950C94BC
:104DF000F62698E0899F90011124622B6093DF02D0
:104E00000E94EF248091DF028595859585950C940D
:104E1000F7261092DF0280E00C94F7269091DF02D3
:104E2000809589238093DF02282F277071F4282F23
:104E3000082E000C330B9217130639F085958595D3
:104E400085950E9410250C94092708956FEF7FEF38
:104E500090E080E00C94593290E080E00E9435327E
:104E600021E08C3E9E4F09F020E0822F089582E0E1
:104E700090E00C94273283E090E00C942732CF939B
:104E800084E090E00E942732C82F81E290E00E94E7
:104E90002732982F8C2FCF910895CF93C92F682F49
:104EA00084E090E00E943B326C2F81E290E0CF9151
:104EB0000C943B32AB01BC018FE090E00C944D327E
:104EC000AB01BC0183E190E00C944D3260E070E0F6
:104ED000CB010C94602760E070E0CB010E945A2760
:104EE0000C9466276CEE7EEF90E080E00E945932D1
:104EF00060E082E090E00E943B3260E083E090E07E
:104F00000E943B321092DB021092DC021092DD0212
:104F10001092DE0260E084E090E00E943B3260E0AC
:104F200081E290E00E943B3260E085E090E00E94E8
:104F30003B3260E086E090E00E943B326FEF87E01A
:104F400090E00E943B3240E050E0BA0188E090E0FF
:104F50000E944D3260E08DE090E00E943B3240E0E4
:104F600050E0BA0188E190E00E944D3260E087E1B4
:104F700090E00E943B3240E050E0BA018CE190E0CA
:104F80000E944D3260E080E290E00E943B320C943F
:104F90006B270C947227682F8EE090E00C943B32C4
:104FA0009C012E5F3F4FAC01485F5F4F80E02417AC
:104FB000350709F40895F90191919F019923B9F3F7
:104FC0008F5FF5CF662349F0FC0132960896219158
:104FD000261729F0E817F907D1F780E0089581E056
:104FE00008959C01FC0132969FEF80E041914617A5
:104FF00051F09F3F19F4411101C0982F8F5F863007
:10500000A9F79F3F09F40895290F311D97FD3A959F
:10501000F90162830895FC013296089621912613C6
:1050200003C0DF0111971C92E817F907B9F708953B
:105030000C94F1270C940B28029626E0FC011192A7
:105040002A95E9F70895089508950C9424280E945C
:10505000252880914B03843049F11092ED0288E1BC
:1050600090E020E40FB6F894A895809360000FBEFE
:105070002093600080E00E9466070E94252883B785
:10508000817F846083BF83B7816083BF7894889574
:1050900083B78E7F83BF0FB6F894A8958091600088
:1050A000886180936000109260000FBE089508959B
:1050B000CF930E9423280E944E0A0E945728C0E0E6
:1050C0008C2F0E94BE09811105C0CF5FC830C1F787
:1050D000CF91089581E0FCCF08950C946C280E9434
:1050E000F7200E947B1C0E9466070C946D281F927B
:1050F0001FB61F9211248F939F93AF93BF938091FC
:10510000ED02811113C08091410390914203A0915F
:105110004303B09144034196A11DB11D8093410307
:1051200090934203A0934303B0934403BF91AF9184
:105130009F918F911F901FBE1F90189582E084BD94
:1051400093E095BD9AEF97BD80936E0008952FB7B9
:10515000F8948091410390914203A0914303B09150
:1051600044032FBF08952FB7F894609141037091C5
:10517000420380914303909144032FBF08959C0103
:105180004FB7F8948091410390914203A09143035B
:10519000B09144034FBF821B930B089578941F92E4
:1051A0001FB61F9211248F939F93AF93BF9380914B
:1051B000410390914203A0914303B09144030196AF
:1051C000A11DB11D8093410390934203A09343031B
:1051D000B0934403BF91AF919F918F911F901FBED9
:1051E0001F90189581E08093E00080E28093D800C2
:1051F0001092C9008FE19EE40197F1F700C0000012
:1052000087E090EBDC018093540390935503A093C7
:105210005603B093570388E19CE00FB6F894A89525
:10522000809360000FBE90936000FFCF0C949E159A
:105230000E944E0A8FE39CE90197F1F700C000003D
:105240000E944E0A80E00E94BE0980FF04C00E94B6
:1052500016290C94F22808950E942C27811102C06F
:105260000E94C9270E9437278093EC020E943F27A3
:1052700090934603809345030E943B27682F70E07C
:1052800090E080E00C948F240F931F9341E050E056
:1052900060E070E08A019B0104C0000F111F221F13
:1052A000331F8A95D2F7C901B8010E948F241F913C
:1052B0000F910C94F7208B3109F46EC040F58B30C0
:1052C00071F078F4863009F450C020F4853059F13B
:1052D00080E00895873009F451C08830C9F781E033
:1052E0000895803109F466C068F48E3089F7909192
:1052F000EC02892F8B7F92FF84608093EC0282FD09
:1053000055C0EDCF863159F3893149F3E1CF8A3267
:1053100049F1B8F4873211F120F48E31C8F28D5181
:105320001EC08932A9F60E94F7202FEF83ED90E38B
:10533000215080409040E1F700C000000E94F22818
:10534000CECF833440F48A3308F03FC0853331F048
:10535000883329F2BDCF833409F0BACF80E00E94B0
:105360004429BDCF0E94C927BACF8091EC02807F2B
:105370008093EC0281E08093EE0208959091EC021C
:10538000892F8E7F90FF81608093EC0280FDA7CFF4
:10539000817F8093EC02A3CF9091EC02892F8D7FC7
:1053A00091FF82608093EC0281FF99CF8091EC02A3
:1053B0008160EFCF9091EC02892F877F93FF886007
:1053C0008093EC0283FDF2CF8ACF8953C8CF80E06F
:1053D00008950C94E729CF93C82F8091EE0288237B
:1053E00031F0813099F01092EE0280E00DC00E9401
:1053F00077268232D1F78C2F0E94E729811116C0BF
:105400008C2F0E945B298170CF9108950E9477268E
:10541000823289F38C2F0E94E929811105C0C431A1
:1054200071F038F4CB3079F781E0EDCF81E090E096
:10543000EACFC93221F0C833B9F380E0E4CF10924B
:10544000EE02FBCF8091F70208950895CF93DF938A
:1054500000D00F92CDB7DEB790914B03943011F589
:1054600089837B836A839093E9008FEF9091E800B2
:10547000815095FD06C095ED9A95F1F700008111D8
:10548000F5CF8091E80085FF0DC050E040E063E07B
:1054900070E0CE0101960E949D2C8091E8008E77ED
:1054A0008093E8000F900F900F90DF91CF910895B7
:1054B000CF93DF93EC010E94802C823011F0843076
:1054C00031F4BE0184E0DF91CF910C94262ADF9164
:1054D000CF910895BC0183E00C94262ACF93DF93EB
:1054E000EC010E94802C823011F0843039F581E08B
:1054F0008093E9008FEF9091E800815095FD06C000
:1055000095ED9A95F1F700008111F5CF8091E800B3
:1055100085FF14C050E040E068E070E0CE010E94DA
:105520009D2C8091E8008E778093E80088E0FE0152
:10553000AFEEB2E001900D928A95E1F7DF91CF9145
:105540000895CF93FC01603221F580914B038430A4
:1055500001F5C091E900CF702091EC00922F91707D
:1055600020FD90E8C92B82E08093E9008091E8005B
:1055700080FF0CC050E040E060E270E0CF010E948C
:105580009D2C8091E8008E778093E800CF70C093C7
:10559000E900CF91089580914A03811109C00E94CA
:1055A0007C2E0E94D92E8091E20084608093E200DC
:1055B000089510924A030895089508950C946F2851
:1055C00042E061EC81E00E94F82D42E261EC84E06F
:1055D0000E94F82D42E261EC82E00E94F82D42E246
:1055E00060EC83E00C94F82D80914D03833009F436
:1055F00061C030F48130D1F1823009F49DC008954A
:105600008A3009F489C08B3009F46FC0893009F001
:1056100050C080914C03813209F04BC080915003FF
:1056200090915103009719F0029709F042C08091C0
:10563000E800877F8093E8008091E80082FF35C012
:105640009091F3008091F200029729F48091F1008B
:105650008B7F813021F48091F1008093F70280915B
:10566000E8008B778093E8000C942C2E80914C03FB
:10567000813AF9F48091E800877F8093E800809177
:10568000500390915103892B61F468E08FEE92E012
:1056900070E00E943B2D8091E8008B778093E800BA
:1056A000089560E090E080E0F3CF80914B0381119A
:1056B000C3CF089580914C03813AD9F7809150036C
:1056C00090915103892BA9F78091E800877F8093FF
:1056D000E8008091E80080FFFCCF80913501809345
:1056E000F1008091E8008E77BDCF80914C0381322C
:1056F00001F78091500390915103892BD1F680914D
:10570000E800877F8093E8000E942C2E80914E0352
:10571000809335010C94F72080914C03813249F637
:105720008091E800877F8093E8000E942C2E809172
:105730004F038093F802089580914C03813A09F059
:10574000B8CF8091E800877F8093E8008091E800DF
:1057500080FFFCCF8091F802C2CFCDB7DEB7A09713
:105760000FB6F894DEBF0FBECDBF84B7877F84BF6E
:105770000FB6F894A89580916000886180936000CE
:10578000109260000FBE80E890E00FB6F89480930E
:105790006100909361000FBE0E94CC1C0E947C2E81
:1057A0000E94D92E8091E20084608093E200789478
:1057B0000E9462310E94D41C8BE291E00E94761C10
:1057C00013E080914B03853039F10E94E01C8091F9
:1057D0004B038430B1F71093E9008091E80082FF19
:1057E000F0CF8091E80090E085FF09C050E040E0F4
:1057F00060E270E0CE0101960E94EC2C91E0809175
:10580000E8008B778093E8009923D9F260E2CE011B
:1058100001960E945616D5CF0E94272880914903F1
:10582000882379F20E945828882359F20E94872CF5
:10583000C8CF0C941B2C292F33272330310521F19D
:1058400068F42130310509F449C02230310509F4EA
:105850004AC090E080E030E020E029C021323105EC
:1058600081F122323105A9F76330710590F7FB0110
:10587000EE0FFF1FEC51FE4F208131816F517E4FA3
:10588000FB01808190E013C099278130910599F048
:10589000009741F08230910589F00397D1F6E6ED4B
:1058A000F9E002C0ECE0FAE0849190E09F01FA0197
:1058B000318320830895EAEFF9E0F6CFECEDF9E0CB
:1058C000F3CF6330710528F6660F771FFB01E651B1
:1058D000FE4F2081318189E090E0E9CF82E190E0C4
:1058E0002BE63AE0E4CF8BE590E020E13AE0DFCF31
:1058F00080914B03843011F482E0089581E0089593
:105900008091F902811102C00C94782C089580E1F5
:1059100089BD82E189BD09B400FEFDCF8091D80028
:105920008F7D8093D8008091E00082608093E000BA
:105930008091E00081FDFCCF0895AF92BF92CF929D
:10594000DF92FF920F931F93CF93DF936C01EB01D4
:105950008A010E944B2EF82E811123C001151105DA
:1059600039F0F80180819181C81BD90BC80ED91E6E
:10597000B12CA12C2097A9F08091E80085FD22C0D0
:105980008091E8008E778093E80001151105A1F061
:10599000F80180819181A80EB91EB182A08285E0B4
:1059A000F82E8F2DDF91CF911F910F91FF90DF90F7
:1059B000CF90BF90AF9008950E944B2E8823D1F2D4
:1059C000F82EEFCFF60181916F018093F1002197BE
:1059D000FFEFAF1ABF0ACECFAF92BF92CF92DF9246
:1059E000FF920F931F93CF93DF936C01EB018A011A
:1059F0000E944B2EF82E811123C00115110539F09C
:105A0000F80180819181C81BD90BC80ED91EB12C19
:105A1000A12C2097A9F08091E80085FD22C08091FB
:105A2000E8008B778093E80001151105A1F0F801DB
:105A300080819181A80EB91EB182A08285E0F82EE6
:105A40008F2DDF91CF911F910F91FF90DF90CF901D
:105A5000BF90AF9008950E944B2E8823D1F2F82E6C
:105A6000EFCF8091F100F60181936F012197FFEF55
:105A7000AF1ABF0ACECFFC0180915203909153031D
:105A800086179707A0F06115710529F49091E80039
:105A90009E779093E80090E06115710551F49111A3
:105AA00008C08091E80082FF34C080E00895BC0106
:105AB000F2CF80914B038823C1F18530C1F18091F1
:105AC000E80083FD30C08091E80082FDEACF80913C
:105AD000E80080FFE1CF8091F3002091F200382FA1
:105AE0006115710519F02830310558F091E0283022
:105AF000310509F090E02091E8002E772093E8002E
:105B0000CBCF81918093F100615071092F5F3F4F9E
:105B1000E7CF80914B03882341F0853041F080919D
:105B2000E80083FFBECF81E0089582E0089583E01E
:105B30000895FC01809152039091530386179707B3
:105B4000A0F06115710529F48091E8008E778093AB
:105B5000E80090E06115710551F4911108C0809141
:105B6000E80082FF35C080E00895BC01F2CF80914B
:105B70004B038823C9F18530C9F18091E80083FD8A
:105B800031C08091E80082FDEACF8091E80080FF7B
:105B9000E1CF8091F3002091F200382F611571055B
:105BA00019F02830310558F091E02830310509F01E
:105BB00090E08091E8008E778093E800CBCF8491CD
:105BC0008093F1003196615071092F5F3F4FE6CF0E
:105BD00080914B03882341F0853041F08091E800AB
:105BE00083FFBDCF81E0089582E0089583E00895AA
:105BF000982F973028F08F708093E90081E0089506
:105C00009093E900242F762F50E0981731F070918F
:105C1000EC002091ED005091F00021FD02C09F5F4B
:105C2000E8CF3091EB003E7F3093EB003091ED00F8
:105C30003D7F3093ED003091EB0031603093EB000D
:105C40007093EC002093ED005093F0002091EE0053
:105C500027FDE5CF80E0089580914C0387FF13C0B6
:105C60008091E80082FF06C08091E8008B778093E6
:105C7000E80004C080914B038111F2CF0895809118
:105C80004B038823D9F38091E80080FFF8CF8091FF
:105C9000E8008E77ECCF2091E4003091E50095E6A6
:105CA000A9012091EC00822F817020FF06C0809115
:105CB000E80080FF06C080E008952091E80022FD02
:105CC0001AC080914B03882389F0853089F0809138
:105CD000EB0085FD0FC02091E4003091E5004217F4
:105CE0005307F9F29150E1F684E0089582E00895B7
:105CF00083E0089581E008950E94EA2E0E94F22E2A
:105D0000E0EEF0E0808181608083E8EDF0E080816A
:105D10008F77808319BCA7EDB0E08C918E7F8C9338
:105D200080818F7E808310924A0308950F931F9382
:105D3000CF93DF930E94EA2E0E94F22EC8EDD0E0AE
:105D400088818F77888388818068888388818F7D28
:105D5000888319BC10924B03109247031092490399
:105D60001092480300EE10E0F80180818B7F808361
:105D700088818160888342E060E080E00E94F82DA5
:105D8000E1EEF0E080818E7F8083E2EEF0E08081C2
:105D900081608083808188608083F80180818E7F2C
:105DA0008083888180618883DF91CF911F910F91DB
:105DB0000895E8EDF0E080818F7E8083E7EDF0E0EC
:105DC00080818160808384E082BF81E080934A0388
:105DD0000C94962EE8EDF0E080818E7F8083109207
:105DE000E20008951092DA001092E10008951F92E7
:105DF0000F920FB60F9211242F933F934F935F93FF
:105E00006F937F938F939F93AF93BF93EF93FF9382
:105E10008091E10082FF0BC08091E20082FF07C009
:105E20008091E1008B7F8093E1000E94613180913D
:105E3000DA0080FF19C08091D80080FF15C08091E2
:105E4000DA008E7F8093DA008091D90080FF96C0BF
:105E500080E189BD82E189BD09B400FEFDCF81E00A
:105E600080934B030E94CB2A8091E10080FF19C0F0
:105E70008091E20080FF15C08091E2008E7F8093C8
:105E8000E2008091E20080618093E2008091D8007E
:105E900080628093D80019BC85E080934B030E94F8
:105EA000DD2A8091E10084FF2BC08091E20084FF15
:105EB00027C080E189BD82E189BD89B5982F9170A5
:105EC00080FFFBCF8091D8008F7D8093D800809198
:105ED000E1008F7E8093E1008091E2008F7E8093CD
:105EE000E2008091E20081608093E20080914703AC
:105EF000882309F449C084E080934B030E94DE2A82
:105F00008091E10083FF29C08091E20083FF25C0DA
:105F10008091E100877F8093E10082E080934B03D2
:105F2000109247038091E1008E7F8093E100809181
:105F3000E2008E7F8093E2008091E2008061809396
:105F4000E20042E060E080E00E94F82D8091F000E5
:105F500088608093F0000E94DC2AFF91EF91BF914E
:105F6000AF919F918F917F916F915F914F913F91F1
:105F70002F910F900FBE0F901F90189519BC109283
:105F80004B030E94D92A70CF8091E30087FD93E0F4
:105F900090934B03B3CF1F920F920FB60F92112421
:105FA0002F933F934F935F936F937F938F939F9321
:105FB000AF93BF93CF93DF93EF93FF93D091E9001B
:105FC000DF708091EC00C82FC17080FDC0E8109296
:105FD000E9008091F000877F8093F00078940E9420
:105FE0000F301092E9008091F00088608093F000FB
:105FF000CD2BCF70C093E900FF91EF91DF91CF914E
:10600000BF91AF919F918F917F916F915F914F91D0
:106010003F912F910F900FBE0F901F9018951F93D7
:10602000CF93DF93CDB7DEB7AA970FB6F894DEBF54
:106030000FBECDBF8CE493E02091F100FC012193D1
:10604000CF01F3E084359F07B9F70E94F42A8091CD
:10605000E80083FF1EC180914C0390914D039A305C
:1060600008F017C1E92FF0E0E75EFC4C0C94B13169
:10607000803899F0823809F00CC1809150038F70FC
:10608000873008F006C18093E9008091EB0085FB22
:10609000882780F91092E90006C08091480390910A
:1060A0004903911182609091E800977F9093E800F6
:1060B0008093F1001092F1008091E8008E77E5C0A6
:1060C000882309F4D3C0823009F0E3C080914E03E5
:1060D0008111D6C0809150038F702FEF280F26308A
:1060E00008F0D7C08093E9002091EB0020FFC8C0E2
:1060F000933031F48091EB0080628093EB00C0C05C
:106100009091EB0090619093EB0021E030E001C0B2
:10611000220F8A95EAF72093EA001092EA00809114
:10612000EB008860EACF8111B4C010914E031F7755
:106130008091E3008078812B8093E3008091E800D8
:10614000877F8093E8000E942C2E8091E80080FFDA
:10615000FCCF8091E30080688093E30082E011111E
:1061600083E080934B0395C08058823008F091C043
:1061700080914E0390914F038C3D23E09207A1F54F
:1061800083E08A838AE289834FB7F894DE0113960D
:1061900020E03EE051E2E32FF0E050935700E4911D
:1061A00020FF03C0E295EF703F5FEF708E2F90E00D
:1061B000EA30C0F0C7968D939D932F5F243159F735
:1061C0004FBF8091E800877F8093E8006AE270E02B
:1061D000CE0101960E943B2D8091E8008B77809341
:1061E000E80057C0C096E7CF60915003709151030B
:1061F000AE014F5F5F4F0E94192CBC01892B09F43F
:1062000048C09091E800977F9093E80089819A8137
:106210000E94992DE1CF8038E1F58091E800877FD9
:106220008093E800809147038093F10045CF81116E
:1062300030C090914E03923060F58091E800877FE6
:106240008093E800909347030E942C2E809147038F
:10625000882311F084E005C08091E30087FDFACF28
:1062600081E080934B030E94E02A13C080914E038B
:10627000813079F481E0933009F080E08093490324
:106280001092E9008091E800877F8093E8000E94E7
:106290002C2E8091E80083FF0AC08091E800877F60
:1062A0008093E8008091EB0080628093EB00AA96D7
:1062B0000FB6F894DEBF0FBECDBFDF91CF911F9117
:1062C00008950895CF9380914B038823A1F0C09146
:1062D000E900CF709091EC00892F817090FD80E8EB
:1062E000C82B1092E9008091E80083FD0E940F30D6
:1062F000CF70C093E900CF910895991B79E004C055
:10630000991F961708F0961B881F7A95C9F78095F4
:106310000895AA1BBB1B51E107C0AA1FBB1FA617EC
:10632000B70710F0A61BB70B881F991F5A95A9F73E
:1063300080959095BC01CD01089597FB072E16F42A
:10634000009407D077FD09D00E94893107FC05D061
:106350003EF4909581959F4F0895709561957F4F7C
:106360000895EE0FFF1F0590F491E02D0994692721
:106370009627692778278727782708958F929F92F5
:10638000AF92BF92CF92DF92EF92FF92CF93DF93C3
:10639000EC01688179818A819B8161157105810594
:1063A000910521F464E279ED8BE597E02DE133EF7F
:1063B00041E050E00E946F3249015A019B01AC015B
:1063C000A7EAB1E40E948E326B017C01ACEEB4EF1F
:1063D000A50194010E949C32DC01CB018C0D9D1D16
:1063E000AE1DBF1DB7FF03C00197A109B048888348
:1063F0009983AA83BB839F77DF91CF91FF90EF9022
:10640000DF90CF90BF90AF909F908F9008950E94A3
:10641000BE31089580E091E00E94BE310895B0E061
:10642000A0E08093000190930101A0930201B0933A
:1064300003010895FC014150504030F001900616D0
:10644000D1F73197CF010895882799270895F999B1
:10645000FECF92BD81BDF89A992780B50895A6E137
:10646000B0E044E050E00C946132A8E1B0E042E0DA
:1064700050E00C946132262FF999FECF92BD81BD78
:10648000F89A019700B4021639F01FBA20BD0FB672
:10649000F894FA9AF99A0FBE08950396272F0E944E
:1064A0003C320E943B32252F0E943C32242F0C9418
:1064B0003C320196272F0E943C320C943B32DC0187
:1064C000CB01FC01F999FECF06C0F2BDE1BDF89AFF
:1064D000319600B40D9241505040B8F70895052E02
:1064E00097FB1EF400940E94863257FD07D00E944D
:1064F000A13207FC03D04EF40C948632509540959F
:10650000309521953F4F4F4F5F4F0895909580955F
:10651000709561957F4F8F4F9F4F08950E94C332B2
:10652000A59F900DB49F900DA49F800D911D1124E7
:106530000895B7FF0C948E320E948E32821B930B0B
:106540000895A1E21A2EAA1BBB1BFD010DC0AA1FB4
:10655000BB1FEE1FFF1FA217B307E407F50720F0CC
:10656000A21BB30BE40BF50B661F771F881F991F47
:106570001A9469F760957095809590959B01AC0190
:10658000BD01CF010895A29FB001B39FC001A39F99
:10659000700D811D1124911DB29F700D811D11245C
:1065A000911D0895F894FFCFD213D913E013E5138A
:1065B000EA13EF13F413F913FE13031408140D1464
:1065C0001114161419141C141F1422142414271443
:1065D0006A1677169E16AA16B516C016C316C616E4
:1065E000C91612171517CC16D016D816E516F216BE
:1065F000F516F8160517DB1EDB1E331F331F851F2C
:10660000081F081F081FA11F2D203C203C20982098
:10661000081F081FA120062106210F210F2111218B
:106620000F210F210F210621062116210F210F21F5
:106630001621383060304931603049319330B43000
:0666400049310B31173156
:106646000100000001F50100F60105F601FB010855
:10665600FC010000000102001000101001191A1BB5
:106666001C1D1E1F2021229230E102222A6E2A259D
:106676002A6A2A582A01E200E900EA00B500B600B3
:10668600B700CD008301CC008A019201940121025A
:10669600230224022502260227022A02B300B4009E
:1066A6006F00700081828332339697343594F5F407
:1066B600F1000000000001020202020606060909B6
:1066C600090909090F0F0F0F0F0F151515181919BD
:1066D60019191919191919192324252525252525C7
:1066E60000FF0100010000FFFF0000010001FF00A4
:1066F600E200E900EA00B500B600B700CD0083016C
:10670600CC008A019201940121022302240225026F
:10671600260227022A02B300B4006F0070008182AD
:1067260083402232D10A7D0A9F0A220A3B0A5B0A6B
:00000001FF
